:020000040800F2
:10300000F8400020013100088D6600085563000873
:103010008966000841330008B5730008000000000D
:1030200000000000000000000000000089680008A7
:10303000773B000800000000C96600083D690008F1
:103040001B3100081B3100081B3100081B31000830
:103050001B3100081B3100081B3100081B31000820
:103060001B3100081B3100081B310008393B0008E8
:103070001B3100081B3100081B3100081B31000800
:103080001B3100081B3100081B3100081B310008F0
:10309000497100081B3100081B3100081B31000872
:1030A0001B3100081B3100081B3100081B310008D0
:1030B0001B3100081B3100081B3100081B310008C0
:1030C0001B3100081B3100081B3100081B310008B0
:1030D0001B3100081B3100081B3100085D7000081F
:1030E0001B3100081B3100081B310008DFF80CD031
:1030F00000F05CF80048004765760008F8400020C2
:103100000648804706480047FEE7FEE7FEE7FEE781
:10311000FEE7FEE7FEE7FEE7FEE7FEE7F5690008EB
:10312000ED300008202A04DB203A21FA02F00021C9
:10313000704721FA02F3D040C2F1200291400843C7
:103140001946704740EA01039B0703D009E008C90C
:10315000121F08C0042AFAD203E011F8013B00F85C
:10316000013B521EF9D27047D2B201E000F8012BA8
:10317000491EFBD270470022F6E710B513460A46F7
:1031800004461946FFF7F0FF204610BD30B505464E
:103190000020034600E05B1C934205D2EC5CC85C57
:1031A000201A01D1002CF6D130BD0000064C074D8D
:1031B00006E0E06840F0010394E807009847103407
:1031C000AC42F6D3FFF796FF108200083082000869
:1031D00070B5044600252068806800F00100F0B159
:1031E0002068806820F001002168886002F07AF988
:1031F00005460EE002F076F9401B022809D9A06AC4
:1032000040F01000A062E06A40F00100E06201209E
:1032100070BD2068806800F001000028EAD100201D
:10322000F6E770B505466C6AA06A00F05000E0B998
:10323000A06A40F40070A0622068806800F46020FA
:10324000B0F5602F0DD1E06858B9A06A20F4807005
:10325000A062A06A00F4805018B9A06A40F0010092
:10326000A062204600F0FAFE03E0206A016B2846C7
:10327000884770BD70B505466C6AA06A40F0400092
:10328000A062E06A40F00400E062204600F0E8FE40
:1032900070BD70B50446656A284600F0E0FE70BD5A
:1032A00038B504460025002000902068806800F0B2
:1032B000010080BB2068806840F0010021688860C0
:1032C000164800681649B0FBF1F0009002E0009843
:1032D000401E009000980028F9D102F003F905463D
:1032E00013E002F0FFF8401B02280ED9A06A40F05C
:1032F0001000A062E06A40F00100E06200BF002020
:1033000084F8240000BF012038BD2068806800F0E8
:1033100001000028E5D00020F6E7000000000020B2
:1033200040420F0010B5044800F066FD0222034938
:10333000014800F087FF10BD940000200400002029
:1033400000BFFEE700B58BB000200690079001207B
:1033500008904FF440400190002002904FF45140FB
:1033600003904FF6FF700490002005900120099013
:1033700001A9154801F026F820B14FF4C07113A03F
:1033800004F01AF801200690002007900120089010
:103390004FF440400190002002904FF451400390C0
:1033A0004FF6FF700490002005900120099001A9BC
:1033B000054801F007F820B140F2951103A003F091
:1033C000FBFF0BB000BD0000582F00202E2E2F5306
:1033D00072632F63616E2E63000000002DE9F041DF
:1033E00004460D46002700260DB9666B00E0A66B6B
:1033F000206800F5D87000EB0510006800F00400AC
:10340000B060B06858B9206800F5D87000EB0510BE
:10341000006840F2FF7101EA505030600AE0206815
:1034200000F5D87000EB051000686FF0604101EA0C
:10343000D0007060206800F5D87000EB05100068BF
:1034400000F00200F060206800F5D87000EB051075
:10345000406800F00F0030613562206800F5D870D8
:1034600000EB05104068C0F30720F061206800F50C
:10347000D87000EB051080683075206800F5D870B2
:1034800000EB05108068010A7175206800F5D8709E
:1034900000EB05108068010CB175206800F5D8704C
:1034A00000EB05108068000EF075206800F5D870FC
:1034B00000EB0510C0683076206800F5D87000EB8E
:1034C0000510C068010A7176206800F5D87000EB1D
:1034D0000510C068010CB176206800F5D87000EBCB
:1034E0000510C068000EF0764DB920202168C86034
:1034F0002068406920F00A002168486108E0202027
:10350000216808612068406920F050002168486106
:1035100094F83C70222F01D0322F05D120684069E9
:1035200020F40F4021684861CDB994F83C0042284E
:1035300004D0622806D072280CD107E0122084F84B
:103540003C000BE0322084F83C0007E0522084F875
:103550003C0003E0012084F83C0000BF19E094F82F
:103560003C00522804D0622806D072280CD107E013
:10357000122084F83C000BE0222084F83C0007E095
:10358000422084F83C0003E0012084F83C0000BFA6
:1035900000BF204601F0DAF90020BDE8F08100000C
:1035A000002037E0002100EB40021C4B23F83210D2
:1035B0004FF4007100EB400203EBC2025180002186
:1035C00000EB400203EBC202918000EB400203EBF0
:1035D000C202D18000EB400203EBC202118100EB7A
:1035E000400203EBC20291720D4901EB402100EB56
:1035F000400203EBC202D160002100EB400203EB6A
:10360000C2021161012100EB400203EBC2021175FD
:10361000411CC8B21628C5DB70470000482D0020A9
:10362000480100202DE9F34F83B0054628890B2877
:103630007EDB0021284603F019FF00907E490098A8
:1036400008700121284603F011FF82467A4981F86B
:1036500001A0009855286CD1BAF1AA0FFBD1288897
:10366000000A88702878C8700221284603F0FEFE00
:10367000064671490E71112E03D0162E01D00C2E64
:103680007ED10321284603F0F1FE80466A4880F887
:1036900005800521284603F0E9FE834604212846DB
:1036A00003F0E4FE0BEB00201FFA80F94FEA19202B
:1036B0006149887181F807900521284603F0D6FEFC
:1036C0000446A8EB040002287DD1298908F10900ED
:1036D000814217DA287D012804D101F003FF286117
:1036E0000020287501F0FEFE2969411A04988142E4
:1036F00005D9297A284603F075FE0120287505B002
:10370000BDE8F08F0120287500270EE0B81DC1B27A
:10371000284603F0ABFE4949C8550846C15D07F18C
:103720000800454A1154781C87B2A742EEDB01E03D
:1037300080E07BE0A01DC1B2284603F097FE4FEA6F
:10374000006BE01DC1B2284603F090FE0BEB004B6E
:1037500004F10800C1B2284603F088FE0BEB002BF1
:1037600004F10900C1B2284603F080FE0BEB000112
:10377000019104F10801304800F028F9029000E0BE
:103780004FE0DDE90110081A41D128882B4B4A4649
:10379000314600F0EFF9A01DC1B2284603F066FEE5
:1037A00004F10801244A5054E01DC1B2284603F038
:1037B0005DFE04F10901204A5054481EC1B228465A
:1037C00003F054FE00E027E004F10A011A4A5054C5
:1037D000481EC1B2284603F049FE04F10B01164A07
:1037E0005054F02104F10C001154401CC2B2124993
:1037F000134803F00BFB08F10900C1B2284603F09F
:10380000F1FD4FF400510F4801F062FE77E701210E
:10381000284603F0E7FD0DE00121284603F0E2FD14
:1038200008E00121284603F0DDFD03E001212846E0
:1038300003F0D8FD00BF62E7DB380020DC37002052
:1038400048000020000C014030B50A4600211CE071
:103850000F4B5B6B14335B5C8588C468635583884E
:103860005B1C9BB283804488A34201DB00238380DE
:1038700003895B1C9BB203814488A34203DD438818
:103880000381012383724B1CD9B29142E0DB30BD2E
:10389000582F00202DE9F047824688461446002C18
:1038A0005DDD2046E11704EB5171C910A4EBC101A5
:1038B0008FB237B90827E11704EB5171C1F3CF0973
:1038C00007E02046E11704EB5171C910491C1FFAAB
:1038D00081F92448006BC0F800A000202149096B41
:1038E000C8602049096B886000261BE008201D493C
:1038F000096B086100250AE0082000FB065018F853
:1039000000101848006B14304155681C85B2082D12
:10391000F2DB0A21134801F059F808B102F0C0FDAA
:10392000701C86B2A9F10100B042DFDC0D48006BCB
:10393000076100250AE0082000FB065018F8001077
:103940000848006B14304155681C85B2BD42F2DB5B
:103950000A21044801F03AF808B102F0A1FDBDE8DF
:10396000F0870000582F002010B5044620684069F9
:1039700020F001002168486194F83C00122805D12C
:103980002068406920F40F402168486194F83C00A9
:10399000422804D0522806D072280CD107E02220F9
:1039A00084F83C000BE0322084F83C0007E0622001
:1039B00084F83C0003E0012084F83C0000BF00BF15
:1039C000204601F05BF9002010BD0000F0B5024672
:1039D0000B460025681E00210FE0565C7040002455
:1039E00007E0060E064F57F8265000026840661C96
:1039F000B4B2042CF5DB4E1CB1B29942EDDBF0BD44
:103A0000587A0008F0B58DB006460F4615460024DA
:103A100004E0305D0BA90855601CC4B2082CF8DB2B
:103A2000002406E020460830305C09A90855601CD7
:103A3000C4B2042CF6DB002405E0FF21201D09AAF6
:103A40001154601CC4B2042CF7DB07AB00223946CA
:103A50000BA803F061FD05AB0022394609A803F06D
:103A60005BFD002405E007A8005D01A90855601C66
:103A7000C4B2082CF7DB002407E005A8015D01AA09
:103A8000204608301154601CC4B2082CF5DB002419
:103A90001CE001A8005D01AA211D515C4840285589
:103AA00001A9201D085C21460831515C4840211DB8
:103AB000685401A920460830085C21460C31515C4D
:103AC0004840214608316854601CC4B2042CE0DB35
:103AD0000DB0F0BD3EB5144A14491548FFF792FFEA
:103AE000002416E0A000C01C0F49085C0106A000DD
:103AF000801C0D4A105C01EB0041A000401C105CD2
:103B000001EB002012F8241008444DF82400601C3A
:103B1000C4B2032CE6DB00F02FF80C2269460548FE
:103B200000F044F93EBD0000283C0020587E00080B
:103B30001C3C002000F4000810B5024801F0F8F821
:103B400010BD0000C400002030B590F840500124A2
:103B5000AC40C56B6C60046863604468102C04D191
:103B60000468A2600468E16003E00468A16004687E
:103B7000E26030BD7047704708B500200B4908600F
:103B80000B4888600120C86001F0F4FA00BF3420BF
:103B90000849C86000BF6946044801F031FA01F0E5
:103BA00087FA642001F018FA08BD00000C3C0020E0
:103BB00000F40008002002400021074AD1610749B3
:103BC000096941F00401054A11611146096941F092
:103BD0004001116170470000383C00200020024085
:103BE0000021074AD1610749096941F00201054AEC
:103BF000116111464861096941F040011161704746
:103C0000383C0020002002400022054BDA61054AC2
:103C1000126942F00102034B1A61018070470000F3
:103C2000383C00200020024038B504466946204652
:103C300001F0E6F908B1012038BD0020FCE70000E2
:103C4000002007490860074888600220C8600020FB
:103C500005490860054888603420C8607047000046
:103C6000E83C002000280008D83C00200030000874
:103C70002DE9F04104460E461746002501F07AFA78
:103C800000BF0EE056F825C0624600232146022000
:103C900001F018FA08B9241D02E00120BDE8F08106
:103CA0006D1CBD4202D203488442EBD901F000FAF8
:103CB0000020F3E7FBFF000800201E49C96801F05F
:103CC000100139B11C49C96941F002011A4AD16198
:103CD00040F010001749C96801F0040139B11649D4
:103CE000C96941F00101144AD16140F00400114951
:103CF000C96901F0010169B10F49C96941F00401C5
:103D00000D4AD16100BF0B49C96921F00101094A7F
:103D1000D16100BF00BF40F20111884206D10549C0
:103D2000C96921F00101034AD16101E00149C8607C
:103D300000BF704700200240383C002070B50446A8
:103D400001F0D0FB054609E0601C38B124B101F058
:103D5000C9FB401BA04201D9032070BD1248C068B6
:103D600000F001000028EFD10F48C06800F02000EB
:103D700020B100BF20200C49C86000BF0A48C068BD
:103D800000F0100048B90848C06900F0010020B9EF
:103D90000548C06800F0040018B1FFF78DFF01204E
:103DA000DBE70020D9E70000002002402DE9F041C8
:103DB00004460E461746002501F0DCF900BF0FE06F
:103DC00056F825C0624600232146022001F07AF908
:103DD00008B9241D03E001F06BF9BDE8F0816D1C0A
:103DE000BD4202D203488442EAD901F061F900BF22
:103DF000F3E70000FBF70008F8B5044600260020B2
:103E0000009000BF94F82400012801D10220F8BDE1
:103E1000012084F8240000BF2046FFF7D9F90646A8
:103E2000002E62D1A06A20F4885040F00200A06207
:103E3000022001F09BFC30490968B1FBF0F0400022
:103E4000009002E00098401E009000980028F9D1F0
:103E50002046FFF725FA2068806840F008002168B6
:103E6000886001F03FFB054611E001F03BFB401B81
:103E70000A280CD9A06A20F0020040F01000A062CD
:103E800000BF002084F8240000BF0120BFE72068A5
:103E9000806800F008000028E7D12068806840F0C2
:103EA00004002168886001F01DFB054611E001F067
:103EB00019FB401B0A280CD9A06A20F0020040F030
:103EC0001000A06200BF002084F8240000BF012081
:103ED0009DE72068806800F004000028E7D1A06A10
:103EE00020F0020040F00100A06200BF002084F832
:103EF000240000BF30468AE70000002038B50246A3
:103F000000230020009000BF92F82400012801D176
:103F1000022038BD012082F8240000BF486807282D
:103F200012D21068406B0C79641E04EB84051F24C8
:103F3000AC40A0430D796D1E05EB85050C68AC40C7
:103F400020431468606327E048680D2812D2106887
:103F5000006B0C79E41F04EB84051F24AC40A043E4
:103F60000D79ED1F05EB85050C68AC402043146806
:103F7000206311E01068C06A0C790D3C04EB8405E5
:103F80001F24AC40A0430D790D3D05EB85050C6861
:103F9000AC4020431468E06208680A2812D3106815
:103FA000C0680C780A3C04EB44050724AC40A043ED
:103FB0000D780A3D05EB45058C68AC40204314683C
:103FC000E0600FE0106800690C7804EB44050724FA
:103FD000AC40A0430D7805EB45058C68AC40204310
:103FE000146820610868102802D00868112827D1B9
:103FF000174C1068A0421ED11068806800F40000C1
:10400000F0B91068806840F400001468A060086887
:10401000102815D10F4800680F4CB0FBF4F000EBEE
:1040200080004000009002E00098401E0090009840
:104030000028F9D104E0906A40F02000906201234A
:1040400000BF002082F8240000BF184661E700008E
:10405000002401400000002040420F0070477047DC
:10406000704700002DE9F041044600270025002696
:10407000A84614B90120BDE8F081A06810B16069BC
:1040800000B100BFA06A30B90020E06284F82400CB
:10409000204600F089F82046FFF79AF80746A06A04
:1040A00000F01000002873D1002F71D1A06A20F415
:1040B000885040F00200A062E16960680843E1684E
:1040C00040EA41000643A068B0F5807F02D0A068B6
:1040D000012802D14FF4807000E0002005436069A0
:1040E000012811D1E06838B9A069401E4FF4006181
:1040F00041EA4030054307E0A06A40F02000A0629A
:10410000E06A40F00100E0622068406820F4694005
:10411000284321684860206880682149084030436E
:1041200021688860A068B0F5807F02D0A06801286F
:1041300002D14FF4807000E00020B0F5807F03D101
:10414000208A401E4FEA00582068C06A20F47000A0
:1041500040EA08002168C862206880681149084068
:10416000B04208D10020E062A06A20F0020040F0D6
:104170000100A06211E0A06A20F0020040F01000EF
:10418000A062E06A40F00100E062012705E0FFE77D
:10419000A06A40F01000A062012738466BE70000DB
:1041A000FDF7E1FFFE0E1FFF10B586B004461C4967
:1041B0002068884232D100BF1A48806940F40070FC
:1041C000184988610846806900F40070019000BFBA
:1041D00000BF03200290039002A9134800F0E2FF01
:1041E000124813490860002048600021104881608F
:1041F0008021C16049000161890041612021816104
:104200000021C16100F062FE18B17E2109A003F017
:10421000D3F800BF06482062446200BF06B010BD5C
:104220000024014000100240000801400800024044
:10423000C40000202E2E2F5372632F6164632E63FF
:10424000000000002DE9F04104460D461646002707
:1042500057492068884203D056492068884205D1D2
:104260005348001D006800F4702000E00020002882
:104270007ED100BF94F82400012802D10220BDE8BD
:10428000F081012084F8240000BF2046FFF708F8E1
:104290000746002F6DD1A06A40F60161884340F4C3
:1042A0008070A06243492068884209D14048001DBF
:1042B000006800F4702008B9012002E0002000E04E
:1042C000012078B1A06A20F48010A06220684068C4
:1042D00000F4806000B3A06A20F4005040F48050E5
:1042E000A06219E0A06A40F48010A0623049206802
:1042F000884203D02F492068884205D12C48001DF0
:10430000006800F4806000E0002028B1A06A20F47A
:10431000005040F48050A062A06A00F4805020B1A8
:10432000E06A20F00600E06201E00020E06200BFE9
:10433000002084F8240000BF1F48216A88621F48BB
:10434000216AC8621E48216A08636FF00200216872
:1043500008602068806840F4807021688860226866
:1043600002F14C0133462A46206A00F0E7FD01E0E5
:104370001AE014E02068806800F46020B0F5602F37
:1043800006D12068806840F4A000216888600CE0B5
:104390002068806840F480102168886005E000BFD4
:1043A000002084F8240000E00127384667E7000079
:1043B0000024014000280140233200089332000805
:1043C0007532000830B5024600230C7D012000FA4A
:1043D00004F31068D0F8000220F47C5001254C6AE8
:1043E00045EA042420431468C4F800021068D0F899
:1043F0001C0298431468C4F81C02C869E8B9106824
:10440000D0F80C0298431468C4F80C02888880B273
:104410008C8940EA0444106800F510704D6940F83A
:104420003540088880B20C8940EA0444106800F5E1
:1044300010704D6900EBC5004460C86901281DD1AA
:104440001068D0F80C0218431468C4F80C0288886D
:1044500080B20C8840EA0444106800F510704D6981
:1044600040F83540888980B20C8940EA04441068DD
:1044700000F510704D6900EBC5004460886938B9DB
:104480001068D0F8040298431468C4F8040206E0E7
:104490001068D0F8040218431468C4F804020869CC
:1044A00038B91068D0F8140298431468C4F814029C
:1044B00006E01068D0F8140218431468C4F8140217
:1044C000086A012806D11068D0F81C021843146845
:1044D000C4F81C021068D0F8000220F00100146833
:1044E000C4F80002002030BD704700002DE9F04103
:1044F0000446002500260027A8462068C068C0F3AF
:10450000001520684069C0F3C0062DB126B148F4FB
:10451000007810202168C86020680069C0F3001589
:1045200020684069C0F380162DB126B148F4806838
:104530001020216808612068406900F0010000280F
:104540003BD0206880687A490840884201D1012028
:1045500000E00020054620688068764908408842CF
:1045600001D1012000E000200646206880687249E1
:104570000840884201D1012000E0002007460DB923
:1045800006B9D7B120688068C0F34005206880680C
:10459000C0F340262068806800F001070DB906B915
:1045A0001FB12046FFF7E0F901E048F400682068F9
:1045B000806862490843216888602068C06800F00C
:1045C000030520684069C0F3400625B11EB10021F3
:1045D0002046FEF703FF2068006900F0030520680D
:1045E0004069C0F3001625B11EB101212046FEF737
:1045F000F5FE206C40EA080020642068806900F025
:10460000010520684069C0F3002620684069C0F3B6
:10461000C0372DB126B11FB1206C40F001002064DD
:1046200020688069C0F3400520684069C0F34026D7
:1046300020684069C0F3C0372DB126B11FB1206C8E
:1046400040F00200206420688069C0F38005206883
:104650004069C0F3802620684069C0F3C0372DB19F
:1046600026B11FB1206C40F00400206420688069EE
:1046700000F0700008B9012000E000200546206825
:104680004069C0F3C02620684069C0F3C03795BBBD
:104690008EB387B32068806900F07005402D1BD071
:1046A00006DC102D09D0202D0CD0302D24D10EE0A9
:1046B000502D16D0602D1FD118E0206C40F008005E
:1046C00020641AE0206C40F01000206415E0206C9B
:1046D00040F02000206410E0206C40F04000206496
:1046E0000BE0206C40F08000206406E0206C40F479
:1046F0008070206401E007E000BF00BF206880698F
:1047000020F0700021688861206C78B10420216855
:104710004860012084F83C002068406948F65B71DD
:104720008843216848612046FFF7DEFEBDE8F0813E
:10473000010000040001000800000110090501004B
:104740002DE9F041044600270026002514B9012078
:10475000BDE8F08194F83C0028B9002084F83D00C1
:10476000204600F0A5F8022084F83C00206800688C
:1047700020F00200216808602068006840F0010015
:104780002168086000F0AEFE06460EE000F0AAFECA
:10479000801B0A2809D9032084F83C0000BF0020B0
:1047A00084F83D0000BF0320D2E72068406800F095
:1047B00001000028EAD02068406800F001000028CD
:1047C00067D0A069012802D145F0800501E025F0FD
:1047D0008005E069012802D145F0400501E025F09F
:1047E0004005206A012802D145F0200501E025F0AE
:1047F0002005606A012802D145F0100501E025F08E
:104800001005A06A012802D145F0080501E025F055
:104810000805E06A012802D145F0040501E025F011
:1048200004052068006820F0FC0028432168086027
:10483000D4E90201084321690843616908436168BA
:10484000491E08432168C8612068006820F0010003
:104850002168086000F046FE06460EE000F042FEC9
:10486000801B0A2809D9032084F83C0000BF0020DF
:1048700084F83D0000BF03206AE72068406800F02C
:1048800001000028EAD12068406800F0010000B96A
:104890000127012F06D100202064012084F83C006C
:1048A000002055E7042084F83C00012050E7000078
:1048B00010B586B004461F492068884237D100BF32
:1048C0001D48C06940F000701B49C8610846C069B6
:1048D00000F00070019000BF00BFC81402900020DB
:1048E0000390049002A9154800F05CFC4FF480503E
:1048F0000290022003900320059002A90F4800F0C7
:1049000051FC00221146142000F0BBFE142000F0E0
:10491000ABFE0B4820630B486063FEF713FD0A48AB
:104920000068406940F0020007490968486106B024
:1049300010BD00000064004000100240000801406B
:104940000801002024010020582F002030B5044623
:10495000606B806810B9606B006940B918480068E6
:10496000406940F0020016490968486130BD0025E1
:1049700019E0606B0068134931F81510884210D1B6
:10498000606B008805EB45010F4A22F83100626B2D
:10499000117C05EB45020C4B03EBC200FEF754FF04
:1049A00003E0681C85B2162DE3DB00BF04480068F5
:1049B000406940F0020002490968486100BFD5E73C
:1049C000582F00202C780008482D00202DE9F041B8
:1049D00004460E46042500272068806800F08060A9
:1049E000B0F1806F0DD02068806800F00060B0F1F9
:1049F000006F06D02068806800F08050B0F1805FC2
:104A00007ED100BF94F83D00012802D10220BDE80C
:104A1000F081012084F83D0000BF94F83C0022287A
:104A200004D0322806D062280CD107E0422084F856
:104A30003C000BE0522084F83C0007E0722084F830
:104A40003C0003E0122084F83C0000BF00BF206857
:104A5000806800F0806008B1002507E02068806869
:104A600000F0006008B1012500E00225206800F593
:104A7000C07000EB0510006800F00101206800F52F
:104A8000C07000EB05100160206B806898B9206849
:104A900000F5C07000EB05100068216BC968226B3F
:104AA000128841EA42510843216801F5C07101EBC7
:104AB0000511086015E0206800F5C07000EB0510D6
:104AC0000068216B8968226B526841EAC201226B3F
:104AD000D26811430143206800F5C07000EB051057
:104AE0000160206B007C00F00F00216B08612068E2
:104AF00000F5C07000EB0510406820F00F0100E0E9
:104B0000B1E0206800F5C07000EB0510416020683E
:104B100000F5C07000EB05104068216B096908437F
:104B2000216801F5C07101EB05114860206BC07D63
:104B30000106206B807D41EA0041206B407D41EA07
:104B40000020216B097D0843216801F5C07101EB4C
:104B500005118860206BC07E0106206B807E41EAD3
:104B60000041206B407E41EA0021206B007E014322
:104B7000206800F5C07000EB0510C160206800F5EA
:104B8000C07000EB0510006840F00101206800F5DE
:104B9000C07000EB0510016000F0A4FC074620E0A7
:104BA000701CF0B126B100F09DFCC01BB04218D9BA
:104BB000032084F83C001DB980202168886009E04A
:104BC000012D03D1E8032168886003E04FF4000061
:104BD0002168886000BF002084F83D0000BF0320EA
:104BE00015E74DB92068806821490840884201D105
:104BF000012016E0002014E0012D09D12068806812
:104C00001C490840884201D101200AE0002008E048
:104C10002068806818490840884201D1012000E0DE
:104C200000200028BCD094F83C00422804D0522830
:104C300006D072280CD107E0222084F83C000BE05B
:104C4000322084F83C0007E0622084F83C0003E056
:104C5000012084F83C0000BF00BF00BF002084F8A2
:104C60003D0000BFD3E6042084F83C000120CEE6DE
:104C7000010000040001000800000110704700005E
:104C800070B50446002594F82100022803D00420C2
:104C9000A063012548E02068006820F00E0021682C
:104CA00008602068006820F00100216808601F4942
:104CB0002068884201D1012026E01C491431206877
:104CC000884201D110201FE018492831206888420D
:104CD00001D1801518E015493C312068884201D186
:104CE000801411E0114950312068884202D14FF4FC
:104CF000803009E00D4964312068884202D14FF4C8
:104D0000801001E04FF080700849083948600120A8
:104D100084F8210000BF002084F8200000BF606BF1
:104D200010B12046616B8847284670BD08000240DC
:104D300070B50446E06B05682068066894F840107A
:104D4000042088402840002846D006F004000028AF
:104D500042D02068006800F0200028B92068006870
:104D600020F004002168086057492068884201D17A
:104D7000042027E0544914312068884201D14020A2
:104D800020E0514928312068884201D1001519E0FE
:104D90004D493C312068884202D14FF4804011E0F7
:104DA000494950312068884202D14FF4802009E0FF
:104DB000454964312068884202D14FF4800001E007
:104DC0004FF08060404908394860E06A00287AD096
:104DD0002046E16A884776E094F840100220884037
:104DE0002840A0B306F0020088B32068006800F0F5
:104DF000200040B92068006820F00A00216808609F
:104E0000012084F8210030492068884201D1022025
:104E100028E02D4914312068884201D1202021E06A
:104E2000294928312068884201D140151AE02649D5
:104E30003C312068884202D14FF4005012E02249F0
:104E400050312068884203D14FF400300AE017E067
:104E50001D4964312068884202D14FF4001001E0FE
:104E60004FF0007018490839486000BF002084F8EE
:104E7000200000BFA06A30B32046A16A884722E024
:104E800094F84010082088402840E0B106F008005F
:104E9000C8B12068006820F00E002168086094F80E
:104EA000401001208840E16B48600120A06384F835
:104EB000210000BF002084F8200000BF206B10B14B
:104EC0002046216B884770BD080002400146002241
:104ED00009B901207047184B0868C01A1423B0FBA9
:104EE000F3F08000086414480838C863022081F891
:104EF00021000868026843F6F0708243D1E901039B
:104F00001843CB6818430B6918434B6918438B69E6
:104F10001843CB6918430243086802600020886286
:104F2000C862086348638863012081F8210000207B
:104F300081F8200000BFCDE7080002402DE9F041D4
:104F400004460D4616461F464FF0000800BF94F871
:104F50002000012802D10220BDE8F081012084F860
:104F6000200000BF94F8210001282CD1022084F8F1
:104F700021000020A0632068006820F00100216863
:104F800008603B46324629462046FEF7DDFDE06AD2
:104F900030B12068006840F00E00216808600BE026
:104FA0002068006820F0040021680860206800681C
:104FB00040F00A00216808602068006840F00100A5
:104FC0002168086006E000BF002084F8200000BFD0
:104FD0004FF002084046BFE770B5044600F082FA81
:104FE00006462546681C10B104480078054400BFF9
:104FF00000F078FA801BA842FAD370BD7C00002034
:105000002DE9F04104460E460127002500BF264841
:10501000007E012802D10220BDE8F0810120224952
:10502000087600BF2068022813D14CF25030FEF7FA
:1050300085FE90BB0120FEF7BFFD4CF25030FEF71D
:105040007DFE07461948006920F0040017490861F1
:1050500023E04CF25030FEF771FEF0B94FF0FF3014
:105060003060A56812E02846FEF7BAFD4CF25030D9
:10507000FEF764FE07460D48006920F002000B4968
:1050800008610FB1356007E005F58065D4E90210CD
:1050900001EB8020A842E6D800BF00BF00200249F3
:1050A000087600BF3846B7E7383C002000200240B1
:1050B0000348006940F08000014908610020704702
:1050C000002002402DE9FE4F05468B4617469846C4
:1050D000012600240020029000BF2448007E012801
:1050E00002D10220BDE8FE8F01202049087600BFD2
:1050F0004CF25030FEF722FE064686BB012D02D14F
:105100000120029006E0022D02D10220029001E06F
:105110000420029000241EE02201B946C2464846FF
:105120005146FDF7FFFF80B20190022000FB04B062
:1051300000900199FEF768FD4CF25030FEF7FEFD3D
:1051400006460B48006920F001000949086106B1D4
:1051500004E0601CC4B202988442DDDB00BF00BFE3
:1051600000200249087600BF3046BBE7383C0020EB
:105170000020024000200849096901F0800151B176
:105180000649054A5160064951601146096901F016
:10519000800101B1012070470020024023016745D2
:1051A000AB89EFCD2DE9F847034600240020002508
:1051B0008446002700226EE14FF0010808FA02F44D
:1051C000D1F8008008EA0400A0427DD1DFF8D0A227
:1051D000D1F80480A8EB0A09D0453AD014DCB8F124
:1051E000030F50D009DCB8F1000F31D0B8F1010F36
:1051F0001CD0B8F1020F49D120E0B8F1110F18D03E
:10520000B8F1120F42D11EE0B9F5881F25D006DC97
:10521000B9F5803F20D0B9F5801F37D11AE0B9F534
:10522000001F18D0B9F5041F30D117E0D1F80CC019
:105230002DE0D1F80C8008F1040C28E0D1F80C80A6
:1052400008F1080C23E0D1F80C8008F10C0C1EE0EA
:1052500000BF00BF00BF00BF00BF00BFD1F8088083
:10526000B8F1000F02D14FF0040C0BE0D1F8088028
:10527000B8F1010F03D14FF0080C1C6102E04FF0B0
:10528000080C5C6103E04FF0000C00E000BF00BFC1
:10529000FF2801D8984601E003F104084646FF289C
:1052A00002D84FEA820803E0A2F108084FEA880812
:1052B0004746D6F800804FF00F0909FA07F928EAA7
:1052C00009080CFA07F900E088E048EA0908C6F87E
:1052D0000080D1F8048008F08058B8F1805F7DD15B
:1052E00000BFDFF8C081D8F8188048F00108DFF867
:1052F000B491C9F81880C846D8F8188008F0010899
:10530000CDF8008000BF00BF4FEAB9384FEA9209DC
:1053100058F829504FEA82784FEA18794FF00F0871
:1053200008FA09F825EA0805DFF87C81434502D12F
:105330004FF0000816E0DFF87481434502D14FF0CA
:1053400001080FE0DFF86881434502D14FF0020801
:1053500008E0DFF86081434502D14FF0030801E027
:105360004FF004084FEA82794FEA197908FA09F8F0
:1053700048EA0505DFF840814FEA920948F82950CC
:10538000D1F8048008F48038B8F5803F0AD1DFF8FE
:105390002C81D8F8008048EA0008DFF82091C9F88D
:1053A000008009E0DFF81481D8F8008028EA0008BE
:1053B000DFF80891C9F80080D1F8048008F40038BB
:1053C000B8F5003F10D1DFF8F48008F10408D8F8F0
:1053D000008048EA0008DFF8E49000E05AE009F1B4
:1053E0000409C9F800800DE0DFF8D08008F1040856
:1053F000D8F8008028EA0008DFF8C09009F1040915
:10540000C9F80080D1F8048008F48018B8F5801F2E
:105410000ED1DFF8A88008F10808D8F8008048EA23
:105420000008DFF8989009F10809C9F800800DE03C
:10543000DFF8888008F10808D8F8008028EA00081A
:10544000DFF8789009F10809C9F80080D1F80480E4
:1054500008F40018B8F5001F0ED1DFF8608008F1DD
:105460000C08D8F8008048EA0008DFF8509009F1ED
:105470000C09C9F800800DE0DFF8408008F10C0845
:10548000D8F8008028EA0008DFF8309009F10C090C
:10549000C9F80080521C102AFFF48EAEBDE8F887D0
:1054A000000011100010024000080140000C0140F3
:1054B00000100140001401400800014000040140B8
:1054C000024693680B400BB1012000E000207047BA
:1054D000C2684A40C26070470AB1016101E00B0432
:1054E00003617047014800687047000074000020A5
:1054F00070B504460CB9012070BD4CF6CC40216853
:10550000086045F2555021680860D4E900104860F1
:105510002168A0688860FFF7E5FF054606E0FFF711
:10552000E1FF401B302801D90320E5E72068C0686F
:105530000028F4D14AF6AA20216808600020DBE7A1
:1055400001464AF6AA200A68106000207047000051
:105550000348006803490978084401490860704716
:10556000740000207C00002010B50848006840F05E
:10557000100006490860032000F0C2F8002000F087
:1055800007F800F02BF8002010BD000000200240BA
:1055900070B504460E4800784FF47A71B1FBF0F014
:1055A0000C490968B1FBF0F5284600F07EFD08B112
:1055B000012070BD102C07D200222146501E00F0A1
:1055C00060F80548046001E00120F2E70020F0E700
:1055D0007C000020000000207800002008B500BFFB
:1055E0001F48806940F001001D49886108468069B4
:1055F00000F00100009000BF00BF032000F080F821
:10560000002211466FF00B0000F03BF8002211461B
:105610006FF00A0000F035F8002211466FF0090023
:1056200000F02FF800221146501F00F02AF8002247
:105630001146101F00F025F800221146901E00F0C0
:1056400020F800221146501E00F01BF800BF05494B
:10565000486820F0E06040F00070486000BF08BD7E
:10566000001002400000014000BF00F01F020121B5
:1056700091404209920002F1E022C2F8001100BFFD
:1056800070472DE9F05F80460D461646002700F072
:10569000FFFF074639462A46334601F00700C0F1AE
:1056A000070ABAF1040F02D94FF0040A01E0C0F171
:1056B000070AD14600F1040ABAF1070F02D24FF0EF
:1056C000000A01E0A0F1030AD4464FF0010A0AFAE9
:1056D00009FAAAF1010A0AEA020A0AFA0CFA4FF0D8
:1056E000010B0BFA0CFBABF1010B0BEA030B4AEAC3
:1056F0000B042146404600F0D3FFBDE8F09F0000B8
:1057000000BF00F00702064B19684FF6FF0319406F
:10571000044B0B4343EA0221014B196000BF704761
:105720000CED00E00000FA0500BF00BF00BF00BFA5
:1057300000BFBFF34F8F00BF00BF00BF0948006824
:1057400000F4E06008490843001D0649086000BFF6
:1057500000BF00BFBFF34F8F00BF00BF00BF00BF3F
:1057600000BFFDE70CED00E00000FA052DE9F04375
:1057700085B006463DA30FCB01AC0FC43FA0006827
:1057800000904FF00008002500270024A146012EBC
:1057900030D0022E58D0102E61D1394844680068AC
:1057A00000F0807000B301A8C4F38341475C04F4A7
:1057B000803070B132484068C0F340401DF800802E
:1057C00004F4803040B12F48B0FBF8F000FB07F53F
:1057D00002E02D4807FB00F52948406800F48000EE
:1057E000B0F5800F01D1A94603E068000321B0FBAA
:1057F000F1F935E02248046A04F44070B0F5807F86
:1058000005D104F0020010B14FF400491BE004F48C
:105810004070B0F5007F07D11948406A00F00200DF
:1058200010B149F640490EE004F44070B0F5407FF5
:1058300007D11348006800F4003010B14FF224493A
:1058400001E04FF000090BE000F0A0F90C494968B5
:10585000C1F38131491C4900B0FBF1F900E000BF00
:1058600000BF484605B0BDE8F08300000203040510
:10587000060708090A0B0C0D0E0F1010010200009C
:105880000010024000127A0000093D00F8B50446FD
:1058900000260025207800F0010000286BD00027AA
:1058A0004348C06900F0805070B900BF4048C069EB
:1058B00040F080503E49C8610846C06900F0805001
:1058C000009000BF00BF01273A48006800F48070D4
:1058D000B0B93848006840F4807036490860FFF776
:1058E00001FE064606E0FFF7FDFD801B642801D996
:1058F0000320F8BD2F48006800F480700028F2D023
:105900002B48006A00F440752DB3A08800F4407065
:10591000A84220D02648006A20F44075012026497C
:105920000860002008602248056205F0010090B17F
:10593000FFF7D8FD064608E0FFF7D4FD801B41F2D3
:105940008831884201D90320D3E71948006A00F062
:1059500002000028F0D01648006A20F44070616808
:10596000084313490862012F04D10846C06920F09A
:105970008050C86100BF207800F00200022807D1E3
:105980000B48406820F44040A1680843084948603B
:10599000207800F01000102807D10548406820F456
:1059A0008000E1680843024948600020A1E7000048
:1059B00000100240007000404004424270B50446AE
:1059C0000D4600266248006800F00700A8420ED28B
:1059D0005F48006820F0070028435D4908600846DA
:1059E000006800F00700A84201D0012070BD2078B7
:1059F00000F00200022807D15648406820F0F0006D
:105A0000A168084353494860207800F0010000284D
:105A10005DD06068012806D14E48006800F400306F
:105A200090B90120E2E76068022806D14948006881
:105A300000F0007040B90120D8E74648006800F047
:105A4000020008B90120D1E74248406820F0030075
:105A5000616808433F494860FFF744FD06466068B7
:105A6000012810D108E0FFF73DFD801B41F288318D
:105A7000884201D90320B9E73648406800F00C009D
:105A80000428F0D123E06068022810D108E0FFF775
:105A900029FD801B41F28831884201D90320A5E706
:105AA0002C48406800F00C000828F0D10FE008E016
:105AB000FFF718FD801B41F28831884201D903208D
:105AC00094E72448406800F00C000028F0D12048FA
:105AD000006800F00700A8420ED91D48006820F0B9
:105AE000070028431A4908600846006800F00700CC
:105AF000A84201D0012079E7207800F004000428B2
:105B000007D11448406820F4E060E1680843114977
:105B10004860207800F00800082808D10D48406847
:105B200020F46050216940EAC1000A49486000F051
:105B30003DF808494968C1F30311074A515CC84060
:105B4000064908600020FFF723FD00204EE7000013
:105B500000200240001002401478000800000020DD
:105B600001480068704700000000002000B5FFF702
:105B7000F7FF04494968C1F30221034A515CC84058
:105B800000BD0000001002402478000800B5FFF7B7
:105B9000E7FF04494968C1F3C221034A515CC84088
:105BA00000BD00000010024024780008F0B585B068
:105BB0000FF26C0C9CE8E01001A8A0E8E0101CA516
:105BC0002D68009500210022002300240020194D9B
:105BD000696801F00C05F5B1042D02D0082D19D12A
:105BE00001E0154819E001ADC1F38346AC5D01F455
:105BF000803555B10F4D6D68C5F340451DF8052042
:105C00000D4D6543B5FBF2F302E00C4D04FB05F3CB
:105C1000184602E000BF084800BF00BF05B0F0BD55
:105C200002030405060708090A0B0C0D0E0F1010DD
:105C3000010200000010024000127A0000093D003D
:105C4000F8B504460025207800F00100002878D03F
:105C5000F848406800F00C0004280CD0F548406873
:105C600000F00C00082811D1F248406800F48030A0
:105C7000B0F5803F0AD1EF48006800F400300028FA
:105C80005FD0606800285CD10120F8BD00BF60686B
:105C9000B0F5803F06D1E748006840F48030E54920
:105CA000086028E0606858B9E248006820F4803055
:105CB000E04908600846006820F4802008601AE087
:105CC0006068B0F5A02F0BD1DA48006840F480205E
:105CD000D84908600846006840F4803008600AE04F
:105CE000D448006820F48030D24908600846006833
:105CF00020F48020086000BF606888B1FFF7F2FBE5
:105D0000054606E0FFF7EEFB401B642801D903209F
:105D1000BBE7C848006800F400300028F2D010E06B
:105D2000FFF7E0FB054606E0FFF7DCFB401B6428BD
:105D300001D90320A9E7BF48006800F4003000281B
:105D4000F2D1207800F00200022857D1B94840680B
:105D500000F00C0050B1B748406800F00C00082873
:105D600018D1B448406800F4803098B9B148006850
:105D700000F0020020B12069012801D0012084E751
:105D8000AC48006820F0F800616940EAC100A94908
:105D9000086033E02069E8B10120A7490860FFF7F7
:105DA000A1FB054606E0FFF79DFB401B022801D939
:105DB00003206AE79F48006800F002000028F2D044
:105DC0009C48006820F0F800616940EAC1009949E8
:105DD000086013E0002098490860FFF783FB054640
:105DE00006E0FFF77FFB401B022801D903204CE7A8
:105DF0009048006800F002000028F2D1207800F0FE
:105E0000080008282DD1A069B8B101208B4908608D
:105E1000FFF768FB054606E0FFF764FB401B02281E
:105E200001D9032031E78348406A00F002000028CE
:105E3000F2D0012000F078FC13E000207F490860D8
:105E4000FFF750FB054606E0FFF74CFB401B02281E
:105E500001D9032019E77748406A00F002000028C2
:105E6000F2D1207800F00400042873D10026714894
:105E7000C06900F0805070B900BF6E48C06940F042
:105E800080506C49C8610846C06900F0805000909D
:105E900000BF00BF01266A48006800F48070B0B9F6
:105EA0006748006840F4807065490860FFF71AFB96
:105EB000054606E0FFF716FB401B642801D90320C6
:105EC000E3E65F48006800F480700028F2D000BF6D
:105ED000E068012806D15748006A40F001005549A2
:105EE000086227E0E06858B95248006A20F00100D3
:105EF000504908620846006A20F00400086219E070
:105F0000E06805280BD14B48006A40F0040049497D
:105F100008620846006A40F0010008620AE045484D
:105F2000006A20F00100434908620846006A20F038
:105F30000400086200BFE068A0B1FFF7D3FA05468D
:105F400009E0FFF7CFFA401B41F28831884202D9BD
:105F500003209AE622E03748006A00F00200002899
:105F6000EFD012E0FFF7BEFA054608E0FFF7BAFAF5
:105F7000401B41F28831884201D9032085E62D4833
:105F8000006A00F002000028F0D1012E05D1294856
:105F9000C06920F080502749C86100BFE069C8B3DC
:105FA0002448406800F00C00082860D0E06902280E
:105FB00048D1002020490866FFF794FA054606E01C
:105FC000FFF790FA401B022801D903205DE619482B
:105FD000006800F000700028F2D1206AB0F5803F20
:105FE00007D11448406820F40030A16808431149E3
:105FF0004860D4E9080108430E49496821F4741146
:1060000008430C49486001200B490866FFF76AFA0B
:10601000054607E02DE0FFF765FA401B022801D98D
:10602000032032E60348006800F000700028F2D038
:106030001FE0000000100240000042428004424283
:106040000070004000200C490866FFF74BFA054637
:1060500006E0FFF747FA401B022801D9032014E6A7
:106060000648006800F000700028F2D101E001202D
:106070000BE6002009E6000000004242001002404A
:10608000042808D14FF0E021096941F004014FF0E4
:10609000E022116107E04FF0E021096921F00401DD
:1060A0004FF0E02211617047704770B504462546F5
:1060B000681EB0F1807F01D301200FE0681E4FF011
:1060C000E02148610F214FF0FF3000F0E9FA002095
:1060D0004FF0E021886107200861002070BD10B5F5
:1060E000FFF7E2FF10BD70472DE9F0470446206836
:1060F00005682068C668206847694FF00008C146F7
:1061000005F00F08B8F1000F0AD105F0200038B1F2
:1061100006F0200020B1204600F025FEBDE8F08703
:10612000B8F1000F6DD007F0010018B906F49070B7
:10613000002866D005F0010030B106F4807018B177
:10614000E06B40F00100E06305F0040030B107F0BF
:10615000010018B1E06B40F00200E06305F00200BE
:1061600030B107F0010018B1E06B40F00400E063CB
:1061700005F0080030B107F0010018B1E06B40F005
:106180000800E063E06B68B305F0200028B106F07A
:10619000200010B1204600F0E6FD20684069C0F301
:1061A0008019E06B00F0080010B9B9F1000F22D09F
:1061B000204600F069FD2068406900F04000B0B161
:1061C0002068406920F0400021684861606B50B150
:1061D0001748616B4863606BFEF752FD10B1606B4E
:1061E000416B88470CE02046FFF77DFF08E0204622
:1061F000FFF779FF04E02046FFF775FF0020E0631A
:106200008CE705F0800030B106F0800018B1204620
:1062100000F0F0FE82E705F0400030B106F04000EB
:1062200018B1204600F040FD78E700BF76E7000097
:106230004D6A000810B504460CB9012010BDA069D4
:1062400000B100E000BF94F8390028B9002084F8BC
:106250003800204600F028F8242084F8390020680F
:10626000C06820F400502168C860204600F0DEFDC0
:106270002068006920F49040216808612068406926
:1062800020F02A00216848612068C06840F400506E
:106290002168C8600020E063202084F8390084F879
:1062A0003A000020CAE7000010B586B00446244931
:1062B0002068884241D100BF2248C06940F4802054
:1062C0002049C8610846C06900F48020019000BFE1
:1062D00000BF08150290022003900320059002A938
:1062E0001948FEF75FFF4FF4006002900020039012
:1062F000049002A91448FEF755FF002211462720FA
:10630000FFF7BFF92720FFF7AFF910480068C06812
:1063100040F480700D490968C8600C480068406905
:1063200040F0010009490968486108480068C068F0
:1063300040F0200005490968C86006B010BD0000A3
:106340000048004000100240000C01409C37002033
:106350007047704700BFFEE7014802490860704778
:106360000030000808ED00E010B5FFF7BBF840F67C
:10637000B83188420DD24FF480611948FFF7A0F878
:10638000044618480470FFF7ADF81749086000206C
:1063900010BD4FF480611248FFF792F8044611488F
:1063A0000078844208D111480078012807D1FFF70E
:1063B00099F80D49086002E000200C490870FFF7C9
:1063C00091F809490968401AB0F57A7F03D901208C
:1063D00006490870DCE7034804700020D8E7000095
:1063E00000080140280000202C0000203000002080
:1063F00070B504460D46FFF775F8A168401AA8422B
:1064000006D9A1882068FFF763F8FFF76BF8A06052
:1064100070BD00000EB51C481C49086081151B4862
:1064200081600121C160002141614FF46021C1619F
:10643000002016494860022114480161FDF712FE50
:1064400018B1452112A000F0B7FF002000900120F4
:1064500001900720029069460C48FDF74FFD18B1E6
:106460004F210BA000F0A8FF012000900220019016
:106470000720029069460548FDF740FD18B15921F3
:1064800003A000F099FF0EBD0024014094000020FD
:106490002E2E2F5372632F6164632E630000000061
:1064A00010B513481349086001151348FFF708F8A1
:1064B000012801D1182000E030200E494860002159
:1064C0000C488160C1604FF440310161002141619D
:1064D00081610121C1610021016241628162C16269
:1064E000FEF72EF918B1692104A000F065FF10BD78
:1064F00000640040582F0020000801402E2E2F532A
:1065000072632F63616E2E630000000008B500BF48
:106510000648406940F00100044948610846406966
:1065200000F00100009000BF00BF08BD0010024055
:1065300000B585B000BF2F48806940F020002D498C
:1065400088610846806900F02000009000BF00BF0D
:1065500000BF0846806940F00400886108468069F1
:1065600000F00400009000BF00BF00BF0846806933
:1065700040F0080088610846806900F0080000903B
:1065800000BF00BF002220211B48FEF7A5FF00220C
:1065900040211948FEF7A0FF002280211648FEF78F
:1065A0009BFF002243F201011448FEF795FFE02013
:1065B0000190012002900220049001A90E48FEF7EC
:1065C000F1FD43F2010001900120029002200490AD
:1065D00001A90A48FEF7E6FD4FF480600190002013
:1065E00002900120039001A90348FEF7DBFD05B0EE
:1065F00000BD00000010024000080140000C0140F6
:1066000010B50848084908600320486040F6C411E6
:1066100005488160FEF76CFF18B13A2103A000F035
:10662000CBFE10BD00300040880000202E2E2F53DE
:1066300072632F697764672E6300000010B50C4801
:106640000C4908604FF4E13048600021094881603E
:10665000C16001610C21416100218161C161FFF7CD
:10666000E9FD18B1452104A000F0A6FE10BD000010
:10667000004800409C3700202E2E2F5372632F7548
:10668000736172742E63000000BFFEE77047000064
:1066900002480068C0F30220704700000CED00E0E3
:1066A00010B5002807DA0A07140E054A00F00F0398
:1066B0001B1FD45403E00A07130E024A135410BDE3
:1066C00018ED00E000E400E07047000010B504465B
:1066D000207801280FD1FEF705FF11490968401AFB
:1066E000B0F57A7F1AD3002201210E48FEF7F4FE9E
:1066F0000020207012E0207802280FD1FEF7F2FE71
:1067000007490968401A40F6B831884206D300228A
:1067100001210448FEF7E0FE0020207010BD0000BB
:1067200060000020000C014008B508490968C9084C
:106730004FF47A72B1FBF2F14143009100BF00BF08
:1067400000994A1E00920029F9D108BD00000020DE
:106750003EB535480568002406E0E00025FA00F063
:1067600032490855601CC4B2042CF6DB2E48001DCB
:106770000568002408E0E00025FA00F0C1B2201D01
:106780002A4A1154601CC4B2042CF4DB2648083099
:106790000568002409E0E00025FA00F0C1B204F128
:1067A0000800224A1154601CC4B2042CF3DB2048B8
:1067B0000568002406E0E00025FA00F01D490855B0
:1067C000601CC4B2042CF6DB1948001D05680024C7
:1067D00008E0E00025FA00F0C1B2201D154A11546E
:1067E000601CC4B2042CF4DB114808300568002496
:1067F00009E0E00025FA00F0C1B204F108000D4AFA
:106800001154601CC4B2042CF3DB6A460A490748E1
:10681000FDF7F8F80C2207496846FCF7B7FC08B901
:1068200000203EBD0120FCE7E8F7FF1F1C3C0020D4
:1068300000F40008283C0020587E000808B5FDF749
:10684000FFF9FEF797FC00BF34200B49C86000BF7A
:106850000A48FDF7E9F90A20FEF7BEFBFEF728FC1F
:1068600007480090012269460648FDF701FA142006
:10687000FEF7B2FB08BD000000200240E83C00200B
:10688000674523010428000870472DE9F043ADF562
:10689000017D81460F46164698464FF4807141A807
:1068A000FCF769FC4FF4807101A8FCF764FC00253B
:1068B000F4B255208DF80401AA208DF805010720B7
:1068C0008DF80601FF208DF807018DF80871A01CD6
:1068D000C0B28DF80901300A8DF80A018DF80B411C
:1068E0002246414643A8FCF72DFC04F1080241A9C9
:1068F00001A8FCF727FC04F1080101A8FDF766F8E0
:106900000546280E04F1080141AA5054C5F3074179
:1069100004F109001154C5F30721401C1154401C17
:106920001554F021401C1154401CC2B241A94846E4
:1069300000F06CFA0DF5017DBDE8F08310B5FEF7AF
:1069400007FEFFF7CCFB10BD10B594B009200A90EC
:106950004FF480300B9000200C9001200E9010908E
:1069600002201190C10312914FF4E01113910AA873
:10697000FFF766F918B1C9211AA000F01DFD0F201C
:10698000059002200690002007904FF48060089048
:1069900000200990022105A8FFF710F818B1D721AF
:1069A00010A000F009FD022001908003039001A8CF
:1069B000FEF76CFF18B1DE210AA000F0FDFCFFF726
:1069C000CFF84FF47A71B0FBF1F42046FFF76DFB7E
:1069D0000420FFF755FB00221146501EFEF751FE22
:1069E00014B010BD2E2E2F5372632F6D61696E2E61
:1069F000630000001148006840F001000F49086082
:106A0000084640680E4908400C494860084600683E
:106A10000C490840094908600846006820F48020B5
:106A200008600846406820F4FE0048604FF41F00EC
:106A30008860C803044908607047000000100240E5
:106A40000000FFF8FFFFF6FE08ED00E070B5054618
:106A50006C6A0020E085E0842046FFF744FB70BDAF
:106A600070B586B006460D4614462846B5F5884FE3
:106A700056D008DCB0F5885F10D06FF40851084498
:106A800000287CD112E0A0F5AA40143800284FD08D
:106A9000A0F58050EC380028F3D171E000234FF4CA
:106AA00088520C214848FFF7F0FE8AE047480078FA
:106AB000D0B9FEF717FD464908602078F02808D1C4
:106AC000012042490870012211464248FEF704FDA8
:106AD0000AE02078F12807D102203C490870012201
:106AE00011463C48FEF7F8FC2078F0280AD1002235
:106AF00040213948FEF7F0FC002280213648FEF79D
:106B0000EBFC0CE02078F12809D101224021324829
:106B1000FEF7E2FC012280212F48FEF7DDFC50E069
:106B2000FFF78CFE012000F058FCFEF7FDFD48E069
:106B30002A482168016061684160A1688160284835
:106B4000E168016021694160264A01462348FCF75B
:106B500059FF2549234802680A6042684A608068F4
:106B600088600F2221A120480C30FCF7EBFA1E4B65
:106B700045F21B520C211448FFF787FE21E01FE06D
:106B8000FCF7A8FF1D4801680091416801918068E9
:106B900002901B4801680391416804918068059048
:106BA0006B4646F218620C210748FFF76EFEC820BC
:106BB000FEF712FA012000F010FCFEF7B5FD00E030
:106BC00000BF00BF06B070BD480000205C00002080
:106BD00060000020000C014000080140DA3900206C
:106BE00064000020E6390020F239002056332E30B0
:106BF0002E315F3230323331303230001C3C0020D5
:106C0000283C002010B50A46C38893421EDB036966
:106C10001B68DB6823F0200304692468E360C388F1
:106C20009B1AC38003691B68DB6843F02003046977
:106C30002468E360114683880B4499B203888B4231
:106C400002DC0388CB1A99B281801CE003691B68BF
:106C5000DB6823F0200304692468E360C188002313
:106C6000C38003691B68DB6843F020030469246860
:106C7000E36083880B4499B203888B4202DC03886B
:106C8000CB1A99B2818010BD0168C96821F4907156
:106C90000268D1600168496921F00101026851610F
:106CA000202180F83A10704710B504462068C0686B
:106CB00020F040002168C860202084F83900204678
:106CC000FFF747FB002010BD00BFC28803889A422F
:106CD000FBD002691268D26822F0800203691B6847
:106CE000DA60C2888AB9026912681268C2F3C012F7
:106CF0005AB102691268516002691268D26842F0A2
:106D0000800203691B68DA6070474388C268D15407
:106D10004288521C92B2428003889A4201D10022DA
:106D20004280C288521CC28002691268D26842F056
:106D3000800203691B68DA6000BFE5E710B5024610
:106D40000B461946D4889C4209DB94880C44A1B2B6
:106D500014888C4204DC14880C1BA1B200E00021D2
:106D6000D468605C10BD70B5044694F83A002228DF
:106D70004AD1A068B0F5805F13D1A56A206940B9F7
:106D800020684068C0F308002880A06A801CA062C8
:106D900019E020684068C0B22880A06A401CA06248
:106DA00011E0206938B920684068C1B2A26A501C5D
:106DB000A062117007E02068406800F07F01A26ABD
:106DC000501CA0621170E08D401E80B2E085C8B9F1
:106DD0002068C06820F020002168C8602068C06872
:106DE00020F480702168C8602068406920F00100AC
:106DF00021684861202084F83A002046FFF7A8FA6D
:106E0000002070BD0020FCE70220FAE7F0B507463D
:106E10000D461646002405E0295D3846FFF754FF6D
:106E2000601CC4B2B442F7DBF0BD00002DE9F041B4
:106E3000044600252068006920F44050E1680843BA
:106E4000216808612169A068084361690843054316
:106E50002068C06841F20C61884328432168C860FB
:106E60002068406920F44070A169084321684861A6
:106E70005F49206888425CD1FEF788FE00EBC001C4
:106E800001EB001061688900B0FBF1F6FEF77EFEB1
:106E900000EBC00101EB001061688900B0FBF1F06C
:106EA0006421B0FBF1F000EBC00101EB0010A6EB98
:106EB0008000322101EB00106421B0FBF1F000F002
:106EC000F006FEF763FE00EBC00101EB0010616805
:106ED0008900B0FBF1F06421B0FBF1F006EB001685
:106EE000FEF754FE00EBC00101EB00106168890061
:106EF000B0FBF1F7FEF74AFE00EBC00101EB00101A
:106F000061688900B0FBF1F06421B0FBF1F000EBA7
:106F1000C00101EB0010A7EB8000322101EB001053
:106F20006421B0FBF1F000F00F003044216888606C
:106F30005BE0FEF71BFE00EBC00101EB0010616897
:106F40008900B0FBF1F6FEF711FE00EBC00101EB8A
:106F5000001061688900B0FBF1F06421B0FBF1F032
:106F600000EBC00101EB0010A6EB8000322101EB29
:106F700000106421B0FBF1F000F0F006FEF7F6FD22
:106F800000EBC00101EB001061688900B0FBF1F07B
:106F90006421B0FBF1F006EB0016FEF7E7FD00EB15
:106FA000C00101EB001061688900B0FBF1F7FEF74A
:106FB000DDFD00EBC00101EB001061688900B0FB52
:106FC000F1F06421B0FBF1F000EBC00101EB001027
:106FD000A7EB8000322101EB00106421B0FBF1F03F
:106FE00000F00F00304421688860BDE8F0810000A7
:106FF00000380140014691F8390021282CD18868D9
:10700000B0F5805F0FD10A6A1088C0F308000B68E2
:107010005860086918B9086A801C086209E0086AA3
:10702000401C086205E00B6A581C086218780B685F
:107030005860C88C401E80B2C88458B90868C068BF
:1070400020F080000B68D8600868C06840F04000FD
:107050000B68D860002070470220FCE710B5054897
:1070600000F00EF8044800F040F80448FFF73CF840
:1070700010BD000034000020480000209C37002094
:1070800008B5026912681268C2F3401262B302695D
:1070900012685268D1B20269126812680022B2B94D
:1070A0004388C268D1544288521C92B242800388FD
:1070B0009A4201DB00224280C288521C92B2C280F6
:1070C00003889A4203DD0288C2800122027200BF57
:1070D0000022009202691268126800920269126826
:1070E0005268009200BF00BF08BD016909680968C5
:1070F000C1F3C01139B301690968C96801F08001A1
:1071000009B36FF08001026912681160C18891B102
:10711000C188491EC1808288C168895C0269126881
:1071200051608188491C89B28180028891420ADBC2
:107130000021818007E001690968C96821F08001A8
:1071400002691268D160704710B50248FDF7CEF9A8
:1071500010BD0000582F00202DE9F34F85B0804668
:10716000B8F806000D287BDB00214046FFF7E6FD5E
:1071700001908B490198087001214046FFF7DEFD20
:107180008246874981F801A00198552869D1BAF152
:10719000AA0FFBD102214046FFF7D0FD804988703D
:1071A00003214046FFF7CAFD7D49C8700846C078F4
:1071B000897800EB012080B2049004214046FFF75B
:1071C000BDFD064676490E71112E03D0162E01D054
:1071D0000C2E7DD105214046FFF7B0FD07467048D3
:1071E000477107214046FFF7A9FD83460621404627
:1071F000FFF7A4FD0BEB00201FFA80F94FEA1920DE
:107200006749887181F8079007214046FFF796FD8E
:107210000446381B02287DD1B8F8061007F10B0090
:1072200081421FDA5F480078012806D1FEF75AF93B
:107230005D49086000205B490870FEF753F95A4920
:107240000968411A0698814207D998F80610404605
:10725000FFF7D8FC01205349087007B0BDE8F08F54
:107260009CE097E001204F49087000250FE005F1F0
:107270000800C1B24046FFF761FD4C494855084639
:10728000415D05F10800464A1154681C85B2A542CB
:10729000EDDB04F10800C1B24046FFF74FFD4FEAB5
:1072A000006B04F10900C1B24046FFF747FD0BEB4C
:1072B000004B04F10A00C1B24046FFF73FFD0BEB63
:1072C000002B04F10B00C1B24046FFF737FD00E090
:1072D0005BE00BEB0001029104F108013048FCF780
:1072E00075FB0390DDE90210081A44D12F4A494684
:1072F0003046FFF7B5FB221D2949091D881EFBF703
:1073000021FF04F10800C1B24046FFF717FDA11D9F
:10731000234A00E034E05054C81CC1B24046FFF795
:107320000DFDE11D1E4A5054C81CC1B24046FFF776
:1073300005FD04F108011A4A5054C81CC1B2404668
:10734000FFF7FCFC04F10901154A5054F02104F147
:107350000A001154421C12490498FCF79BFA07F1E9
:107360000B00C1B24046FFF74DFC4FF400511048EE
:10737000FEF7AEF871E701214046FFF743FC0DE050
:1073800001214046FFF73EFC08E001214046FFF79F
:1073900039FC03E001214046FFF734FC00BF5CE705
:1073A0000C3B0020700000206C0000200D3A0020F3
:1073B000000C014000BFFEE700BFFEE702E008C886
:1073C000121F08C1002AFAD170477047002001E05F
:1073D00001C1121F002AFBD1704700F0010181F3A7
:1073E0001388704710B50A46038993421EDB1E4B73
:1073F0001B685B6923F002031B4C246863610389EB
:107400009B1A0381184B1B685B6943F00203164CFF
:10741000246863611146C3880B4499B243888B4248
:1074200002DC4388CB1A99B2C1801CE00E4B1B686A
:107430005B6923F002030C4C24686361018900231B
:107440000381094B1B685B6943F00203064C246807
:107450006361C3880B4499B243888B4202DC438842
:10746000CB1A99B2C18010BD582F002010B502462A
:107470000B46194614899C4209DBD4880C44A1B2FE
:1074800054888C4204DC54880C1BA1B200E000211B
:10749000D468605C10BD00007FB50646002404E09F
:1074A000305D18490855601CC4B2082CF8DB38233D
:1074B000154A02A9304600F085F900241EE0002597
:1074C00004E002A800F03EF9681CC5B20F48005D58
:1074D000A842F6DC40230E4A694602A800F072F981
:1074E000002507E06846405DE1000A4A89184855D2
:1074F000681CC5B2082DF5DB601CC4B2102CDEDBA5
:107500007FBD00007D000020207F0008F88100087A
:10751000587F0008583C0020FFB587B00F46002573
:107520000AE0785D3349495D884203D03846FFF769
:10753000B3FF0725681CC5B2082DF2DB40232E4A95
:1075400005A9079800F03EF9012538E0002405E080
:1075500005A8005D03A90855601CC4B2082CF7DB20
:107560000998002805D1681EC000244940180090E1
:1075700005E01020401BC000204940180090002466
:1075800006E003A9201D085C05A90855601CC4B2CB
:10759000042CF6DB01AA05A9009800F033F80024BA
:1075A00009E003A8005D01A9095D484005AA211D65
:1075B0005054601CC4B2042CF3DB681CC5B2112DFE
:1075C000C4DB6846067D017E01750676467D417EF8
:1075D00041754676867D817E81758676C67DC17EC3
:1075E000C175C6764023064A05A80A9900F0EAF854
:1075F0000BB0F0BD7D000020607E0008583C0020EC
:10760000A07E0008F0B587B005460E461746402319
:10761000114A05A9304600F0D5F8002411E005A86C
:10762000005D295D48408006800E03A90855A00131
:107630000A49401803A9095D405C01A90855601C6E
:10764000C4B2082CEBDB2023054A394601A800F020
:10765000B9F807B0F0BD0000987F0008F87F000877
:10766000D87F0008FEF778FEFDF77EFFFFF76CF984
:10767000FEF75EFFFEF74AFFFEF7CCFEFEF710FFB7
:10768000FEF7BEFFFEF7DAFFFBF78AFFFBF74AFEC5
:10769000C820FDF7A1FC22484088B0F57A7F04DAC3
:1076A000012220211F48FDF717FFFFF751F81E495F
:1076B000087033E01D48FDF743FFC8211C48FFF761
:1076C0004BFD1C48FFF702F817480078C0B90024AA
:1076D00000BF09E004EB4401174A02EBC100C821D6
:1076E000FBF7A0FF601C84B2162CF3DBFA211348D1
:1076F000FEF77EFE4FF47A711148FEF779FE07E03F
:1077000064210E48FEF774FE64210D48FEF770FEFA
:10771000FEF72AFE012801D1FEF7C2FECAE70000EB
:1077200004000020000801407100002088000020B3
:10773000340000205C000020482D002008000020BC
:10774000180000200CB5002104E0425C6B465A543E
:107750004A1CD1B20829F8DB002112E0425C520633
:10776000120E425406290ADA6B464A1C9A5C8023A0
:107770001A40802A03D1425C01231A4342544A1C16
:10778000D1B20729EADB6A46127880231A40002A20
:1077900004D0C27810231A43C27003E0C2781023C9
:1077A0009A43C2706A46D27808231A40002A04D04D
:1077B000827901231A43827103E0827952085200D0
:1077C00082710CBDFFB5124C002000BF002605469B
:1077D000401C4E550828F9DB002000BF1378521CCE
:1077E000DE10009DAD5D5E07760FA65D3540002D75
:1077F00007D0C5104D5D4607760FA65D3543C61010
:107800008D55451C2846039EB542E7DBFFBD0000B1
:1078100008820008000000000000000001020304CC
:107820000607080900000000010203041007120700
:107830001307140715071506200721072307240738
:10784000250730073107320734073507350640076B
:1078500041074207430745070000211042206330DB
:107860008440A550C660E770088129914AA16BB198
:107870008CC1ADD1CEE1EFF1311210027332522240
:10788000B5529442F772D662399318837BB35AA3E8
:10789000BDD39CC3FFF3DEE3622443342004011410
:1078A000E664C774A44485546AA54BB52885099538
:1078B000EEE5CFF5ACC58DD55336722611163006E0
:1078C000D776F6669556B4465BB77AA71997388788
:1078D000DFF7FEE79DD7BCC7C448E5588668A778A0
:1078E0004008611802282338CCC9EDD98EE9AFF9D8
:1078F000488969990AA92BB9F55AD44AB77A966A80
:10790000711A500A333A122AFDDBDCCBBFFB9EEB27
:10791000799B588B3BBB1AABA66C877CE44CC55C4F
:10792000222C033C600C411CAEED8FFDECCDCDDD77
:107930002AAD0BBD688D499D977EB66ED55EF44E1F
:10794000133E322E511E700E9FFFBEEFDDDFFCCFC7
:107950001BBF3AAF599F788F8891A981CAB1EBA11B
:107960000CD12DC14EF16FE18010A100C230E32097
:107970000450254046706760B9839893FBA3DAB33F
:107980003DC31CD37FE35EF3B1029012F322D232E7
:107990003542145277625672EAB5CBA5A89589850F
:1079A0006EF54FE52CD50DC5E234C324A014810437
:1079B0006674476424540544DBA7FAB79987B897DF
:1079C0005FE77EF71DC73CD7D326F2369106B01687
:1079D00057667676154634564CD96DC90EF92FE99F
:1079E000C899E9898AB9ABA94458654806782768D7
:1079F000C018E1088238A3287DCB5CDB3FEB1EFB7F
:107A0000F98BD89BBBAB9ABB754A545A376A167A26
:107A1000F10AD01AB32A923A2EFD0FED6CDD4DCD4E
:107A2000AABD8BADE89DC98D267C076C645C454C76
:107A3000A23C832CE01CC10C1FEF3EFF5DCF7CDF1E
:107A40009BAFBABFD98FF89F176E367E554E745EC6
:107A5000932EB23ED10EF01E00000000B71DC104EF
:107A60006E3B8209D926430DDC7604136B6BC51778
:107A7000B24D861A0550471EB8ED08260FF0C922F0
:107A8000D6D68A2F61CB4B2B649B0C35D386CD3158
:107A90000AA08E3CBDBD4F3870DB114CC7C6D04824
:107AA0001EE09345A9FD5241ACAD155F1BB0D45B00
:107AB000C2969756758B5652C836196A7F2BD86E68
:107AC000A60D9B6311105A6714401D79A35DDC7DE0
:107AD0007A7B9F70CD665E74E0B6239857ABE29CCC
:107AE0008E8DA191399060953CC0278B8BDDE68F00
:107AF00052FBA582E5E66486585B2BBEEF46EABAE8
:107B00003660A9B7817D68B3842D2FAD3330EEA9DF
:107B1000EA16ADA45D0B6CA0906D32D42770F3D043
:107B2000FE56B0DD494B71D94C1B36C7FB06F7C377
:107B30002220B4CE953D75CA28803AF29F9DFBF66F
:107B400046BBB8FBF1A679FFF4F63EE143EBFFE557
:107B50009ACDBCE82DD07DEC77708634C06D47306F
:107B6000194B043DAE56C539AB0682271C1B432377
:107B7000C53D002E7220C12ACF9D8E1278804F16EF
:107B8000A1A60C1B16BBCD1F13EB8A01A4F64B0557
:107B90007DD00808CACDC90C07AB9778B0B6567C23
:107BA00069901571DE8DD475DBDD936B6CC0526FFF
:107BB000B5E6116202FBD066BF469F5E085B5E5A67
:107BC000D17D1D576660DC5363309B4DD42D5A49DF
:107BD0000D0B1944BA16D84097C6A5AC20DB64A893
:107BE000F9FD27A54EE0E6A14BB0A1BFFCAD60BBFF
:107BF000258B23B69296E2B22F2BAD8A98366C8EE7
:107C000041102F83F60DEE87F35DA9994440689DDE
:107C10009D662B902A7BEA94E71DB4E0500075E442
:107C2000892636E93E3BF7ED3B6BB0F38C7671F776
:107C3000555032FAE24DF3FE5FF0BCC6E8ED7DC26E
:107C400031CB3ECF86D6FFCB8386B8D5349B79D156
:107C5000EDBD3ADC5AA0FBD8EEE00C6959FDCD6DC4
:107C600080DB8E6037C64F643296087A858BC97E7A
:107C70005CAD8A73EBB04B77560D044FE110C54BEA
:107C8000383686468F2B47428A7B005C3D66C1585A
:107C9000E4408255535D43519E3B1D252926DC213E
:107CA000F0009F2C471D5E28424D1936F550D83202
:107CB0002C769B3F9B6B5A3B26D6150391CBD40762
:107CC00048ED970AFFF0560EFAA011104DBDD014E2
:107CD000949B93192386521D0E562FF1B94BEEF546
:107CE000606DADF8D7706CFCD2202BE2653DEAE602
:107CF000BC1BA9EB0B0668EFB6BB27D701A6E6D3E2
:107D0000D880A5DE6F9D64DA6ACD23C4DDD0E2C0E1
:107D100004F6A1CDB3EB60C97E8D3EBDC990FFB91D
:107D200010B6BCB4A7AB7DB0A2FB3AAE15E6FBAA79
:107D3000CCC0B8A77BDD79A3C660369B717DF79F69
:107D4000A85BB4921F4675961A163288AD0BF38C59
:107D5000742DB081C330718599908A5D2E8D4B59F9
:107D6000F7AB085440B6C95045E68E4EF2FB4F4A79
:107D70002BDD0C479CC0CD43217D827B9660437FE9
:107D80004F460072F85BC176FD0B86684A16476C59
:107D900093300461242DC565E94B9B115E565A153D
:107DA00087701918306DD81C353D9F0282205E0601
:107DB0005B061D0BEC1BDC0F51A69337E6BB523361
:107DC0003F9D113E8880D03A8DD097243ACD5620E1
:107DD000E3EB152D54F6D4297926A9C5CE3B68C10D
:107DE000171D2BCCA000EAC8A550ADD6124D6CD201
:107DF000CB6B2FDF7C76EEDBC1CBA1E376D660E7E1
:107E0000AFF023EA18EDE2EE1DBDA5F0AAA064F4E0
:107E1000738627F9C49BE6FD09FDB889BEE0798D1C
:107E200067C63A80D0DBFB84D58BBC9A62967D9E78
:107E3000BBB03E930CADFF97B110B0AF060D71AB68
:107E4000DF2B32A66836F3A26D66B4BCDA7B75B858
:107E5000035D36B5B440F7B121402324255E262AC0
:107E600039312921191109013B332B231B130B0332
:107E70003D352D251D150D053F372F271F170F07E2
:107E800038302820181008003A322A221A120A0222
:107E90003C342C241C140C043E362E261E160E06D2
:107EA00027072F0F37173F1F26062E0E36163E1EAA
:107EB00025052D0D35153D1D24042C0C34143C1CBA
:107EC00023032B0B33133B1B22022A0A32123A1ACA
:107ED00021012909311139192000280830103818DA
:107EE0002122232425262728292A2B2C2D2E2F300A
:107EF0003132333435363738393A3B3C3D3E3F40FA
:107F00000102030405060708090A0B0C0D0E0F10E9
:107F10001112131415161718191A1B1C1D1E1F20D9
:107F20003830282018100800393129211911090189
:107F30003A322A221A120A023B332B233E362E26CD
:107F40001E160E063D352D251D150D053C342C2421
:107F50001C140C041B130B0300000D04100A170063
:107F6000000002091B0E051400001607120B03196E
:107F700000000F01061A130C00002836331E242EB1
:107F800000001D2F27322C2000002B3430263721F3
:107F900000002D1F2931231C00001F0400010203D3
:107FA00000000308040506070000070C08090A0B77
:107FB00000000B100C0D0E0F00000F141011121307
:107FC00000001318141516170000171C18191A1B97
:107FD00000001B001C1D1E1F1F0E272C3C173724E2
:107FE000041E2E350C253E15050F2F1D3F36061499
:107FF000261C3D0D2D1607340E040D01020F0B0833
:10800000030A060C05090007000F07040E020D0104
:108010000A060C0B0905030804010E080D06020BE5
:108020000F0C0907030A05000F0C080204090107D9
:10803000050B030E0A00060D0F01080E060B0304C4
:108040000907020D0C00050A030D04070F02080EB4
:108050000C00010A06090B05000E070B0A040D01AE
:1080600005080C060903020F0D080A01030F04029C
:108070000B06070C00050E090A00090E06030F0582
:10808000010D0C070B0402080D0700090304060A82
:108090000208050E0C0B0F010D060409080F030062
:1080A0000B01020C050A0E07010A0D00060908075C
:1080B000040F0E030B05020C070D0E030006090A40
:1080C000010208050B0C040F0D080B05060F000339
:1080D0000407020C010A0E090A0609000C0B070D21
:1080E0000F01030E05020804030F00060A010D0824
:1080F0000904050B0C07020E020C0401070A0B060B
:108100000805030F0D000E090E0B020C04070D01EC
:1081100005000F0A030908060402010B0A0D0708EF
:108120000F090C050603000E0B080C07010E020DCB
:10813000060F00090A0405030C010A0F09020608CC
:10814000000D03040E07050B0A0F0402070C0905B6
:1081500006010D0E000B0308090E0F0502080C03A3
:108160000700040A010D0B060403020C09050F0A9F
:108170000B0E01070600080D040B020E0F00080D80
:10818000030C0907050A06010D000B070409010A83
:108190000E03050C020F080601040B0D0C03070E5D
:1081A0000A0F060800050902060B0D0801040A075C
:1081B0000905000F0E02030C0D020804060F0B0147
:1081C0000A09030E05000C07010F0D080A03070436
:1081D0000C05060B000E0902070B0401090C0E0228
:1081E00000060A0D0F03050802010E07040A080D18
:1081F0000F0C09000305060B010102020202020234
:108200000102020202020201804020100804020161
:10821000308200080000002088000000BC730008C5
:10822000B88200088800002070400000CC7300086D
:1082300000A24A0400000000000C014000100000F1
:108240000000000000000000000C014000200000C1
:10825000000000000000000001000000000000001D
:108260000100000000040000000000000000000009
:108270009C2F00209C37002000040000000000001C
:10828000000000009C3300209C370020000000000C
:1082900000000000000000000000000000000000DE
:1082A00001010000000000001000000001000000BB
:0882B0000000000000000000C6
:04000005080030EDD2
:00000001FF
